:100000000C945C000C94D1060C94FE060C948400B5
:100010000C9484000C9484000C9484000C94840050
:100020000C9484000C9484000C9484000C94840040
:100030000C9484000C9484000C9484000C94840030
:100040000C942B070C9484000C9499090C94840054
:100050000C9484000C9484000C9484000C94840010
:100060000C9484000C948400000024272A000025AE
:10007000282B000023262904040404040404040299
:100080000202020202030303030303010204081035
:100090002040800102040810200102040810200002
:1000A0000000070002010000030406000000000039
:1000B00000000000F401BD0511241FBECFEFD4E005
:1000C000DEBFCDBF11E0A0E0B1E0E2EDF4E102C09F
:1000D00005900D92AA33B107D9F712E0AAE3B1E077
:1000E00001C01D92A131B107E1F710E0C8EBD0E0EB
:1000F00004C02297FE010E945B0AC43BD107C9F7E6
:100100000E94B6050C94670A0C940000FC01108252
:100110008FEF81831382128282E2848386E9858352
:10012000178216820895EF92FF920F931F93CF9339
:10013000DF93EC019B0177FF03C020E030E005C0B6
:10014000653B710514F024EB30E02983EC806D8170
:1001500070E06E197109882777FD8095982F982F88
:10016000872F762F662730E040E050E00E94D609C6
:1001700024EB30E040E050E00E942A0AFF2400E037
:1001800010E0102F0F2DFE2CEE24E20EF31E041FA4
:10019000151FC801B70120E430E040E050E00E94A4
:1001A0002A0A3B832A83DF91CF911F910F91FF9001
:1001B000EF9008955F926F927F928F929F92AF928D
:1001C000BF92CF92DF92EF92FF920F931F93DF9334
:1001D000CF93CDB7DEB76DB67EB6ADB65EB60E9434
:1001E0009B0720913C0130913D0140913E0150918F
:1001F0003F01621773078407950750F02C5E3F4F4D
:100200004F4F5F4F621773078407950708F4AFC01D
:1002100060933C0170933D0180933E0190933F01B8
:10022000E0913A01F0913B01BB2408C082819381A7
:10023000892B09F0B3940680F781E02D3097B1F750
:10024000BB2009F494C08B2D90E0880F991F2DB727
:100250003EB7281B390B0FB6F8943EBF0FBE2DBF1B
:10026000CDB6DEB60894C11CD11CA0913A01B09164
:100270003B0120E013C012968D919C911397892B1E
:1002800049F0E22FF0E0EE0FFF1FEC0DFD1DB183F2
:10029000A0832F5F16960D90BC91A02D109759F753
:1002A0002CC0812F90E07C01EE0CFF1CEC0CFD1C9F
:1002B000D7016D917C91FC013197EE0FFF1FEC0D82
:1002C000FD1D40815181DB0112962D913C911397C8
:1002D000DA0112968D919C9113972817390730F403
:1002E000D7014D935C937183608301E01F5F1B1501
:1002F000C0F2002311F410E011C011E000E0F7CFCC
:10030000E12FF0E0EE0FFF1FEC0DFD1D0190F081DD
:10031000E02D61E080810E9491081F5F1B1580F332
:10032000F6B4EE2400E010E08F2C99241EC0EE2DD0
:10033000F0E0EE0FFF1FEC0DFD1D0190F081E02DB0
:1003400022813381280D391D86B58F1510F4005098
:100350001F4FF82EC8018F0D911D28173907A0F7E0
:1003600060E080810E949108E394EB1400F38A2DF1
:10037000952D9C010FB6F8943EBF0FBE2DBF0FB652
:10038000F8947EBE0FBE6DBECF91DF911F910F918D
:10039000FF90EF90DF90CF90BF90AF909F908F90A5
:1003A0007F906F905F9008950F931F938C01FC01D5
:1003B00060838FEF81831382128280913A01909142
:1003C0003B019783868310933B0100933A0160E0E1
:1003D00080810E94910861E0F80180810E94730889
:1003E00081E01F910F91089580E491E00E948600C2
:1003F00088E491E00E94860080E591E00E948600FA
:10040000089540E05BE460E070E08BE791E00E94DB
:10041000CE0564E670E080E090E00E94A90760915C
:1004200021017091220180E591E00E94D40160E0F9
:10043000809131010E94730861E0809132010E9435
:10044000730861E0809132010E94910861E080911F
:100450002F010E9491086DE570E080E591E00E9417
:10046000930061E080911B010E94730861E080911C
:100470001D010E94730861E080911F010E947308B2
:1004800060E08EE00E94730860E08FE00E947308D5
:1004900060E080E10E94730860E081E10E947308DF
:1004A00061E08EE00E94910861E08FE00E94910877
:1004B00061E080E10E94910861E081E10E94910881
:1004C00060E070E080911D010E941B088091230173
:1004D0000E94DC08892B39F081E090E090935B0169
:1004E00080935A0104C010925B0110925A018091CE
:1004F00025010E94DC08892B39F082E090E090937E
:100500005D0180935C0104C010925D0110925C015A
:10051000809127010E94DC08892B39F084E090E06B
:1005200090935F0180935E0104C010925F0110926E
:100530005E01809129010E94DC08892B39F088E056
:1005400090E0909361018093600104C0109261017A
:100550001092600180915C0190915D0120915A019F
:1005600030915B01820F931F20915E0130915F01FA
:10057000820F931F2091600130916101820F931FC0
:10058000909359018093580160E071E08BE791E00E
:100590000E94D30560915801709159018BE791E059
:1005A0000E94C10660E080911F010E94910861E0F5
:1005B00080912F010E94910860E080912B010E94A0
:1005C000910860E080912D010E9491080895EF92BA
:1005D000FF921F93CF93DF937C0160E08091320103
:1005E0000E94910884E590E00E94D30711E0C8E0E2
:1005F000D0E0812F90E08E219F21892B11F061E0C6
:1006000001C060E0809132010E94910884E590E091
:100610000E94D307110F219761F761E080913201A9
:100620000E94910884E590E00E94D307DF91CF916A
:100630001F91FF90EF90089582E090E00E945F0A82
:100640000E94E702089581E090E00E945F0A0E9404
:10065000E7020895EF92FF920F931F930E94DA0032
:100660008BE791E00E94CB05882309F45CC08BE7FF
:1006700091E00E94C805282F80936201803F39F4E1
:1006800081E090E09093700180936F010BC08091A6
:100690006F0190917001019749F4809179019091D7
:1006A0007A01019690937A01809379018091790182
:1006B00090917A0182309105B1F4422F50E09A0175
:1006C000E4E035952795EA95E1F7809158019091FE
:1006D000590128173907F9F44F7050705093780179
:1006E0004093770120C00397F1F4422F50E09A0124
:1006F00074E0359527957A95E1F7809158019091AE
:1007000059012817390739F44F705070509372010E
:100710004093710108C01092700110926F01109205
:100720007A01109279018091790190917A01039771
:1007300009F0B1C180916F0190917001019709F0AA
:10074000AAC110927A011092790110927001109250
:100750006F016AE070E080E090E00E94A90780915C
:100760007701909178018430910509F43EC185307C
:10077000910594F48130910509F498C08230910577
:100780001CF4892BC9F087C18230910509F408C196
:10079000039709F080C112C18630910509F458C150
:1007A000863091050CF42DC18730910509F45CC1A8
:1007B000099709F070C164C1809171019091720133
:1007C0008730910509F449C088309105ACF4833035
:1007D0009105B9F1843091054CF48130910539F1DE
:1007E000823091055CF5892BF9F050C08530910578
:1007F00071F106977CF528C08B309105B9F18C30EA
:10080000910534F48930910559F10A9764F525C0B2
:100810008D30910589F18D3091055CF18E30910517
:1008200071F10F9799F52EC084EB90E002C084E639
:1008300090E0909374018093730128C08AE590E062
:10084000F8CF80E590E0F5CF86E490E0F2CF8CE33E
:1008500090E0EFCF82E390E0ECCF86E290E0E9CF4A
:1008600089E190E0E6CF8FE090E0E3CF8AE090E08E
:10087000E0CF88E090E0DDCF86E090E0DACF83E063
:1008800090E0D7CF109274011092730160E08091D4
:100890002F010E9491088091730190917401843B13
:1008A00091050CF4F8C00E941C03F5C08091710101
:1008B000909172018730910509F447C08830910505
:1008C000ACF483309105A9F1843091054CF481306A
:1008D000910549F1823091054CF5892BF9F050C012
:1008E0008530910561F106976CF526C08B30910536
:1008F000A9F18C30910534F48930910549F10A97BA
:1009000054F523C08D30910579F18D3091054CF16E
:100910008E30910561F10F9799F52CC010927601F8
:10092000109275012DC083E090E026C086E090E033
:1009300023C088E090E020C08AE090E01DC08FE0F6
:1009400090E01AC089E190E017C086E290E014C000
:1009500082E390E011C08CE390E00EC086E490E06A
:100960000BC080E590E008C08AE590E005C084E611
:1009700090E002C084EB90E0909376018093750143
:1009800060E080912F010E94910880917501909103
:100990007601843B91050CF47EC00E9423037BC04A
:1009A0008091710190917201019711F461E001C091
:1009B00060E080911F010E9491086DC060E080910D
:1009C0002F010E94910880917101909172012BE09A
:1009D00030E0829FB001839F700D929F700D1124B3
:1009E00080E591E00E94930056C080917101909142
:1009F0007201019711F461E001C060E080912D0166
:100A0000DACF209171013091720121303105A9F4C2
:100A100084E690E090936C0180936B0130936E01BB
:100A200020936D010E949B0760936701709368019A
:100A30008093690190936A012EC010926E0110920A
:100A40006D0160E070E080911D010E941B0823C0D1
:100A50008091710190917201019711F461E001C0E0
:100A600060E080911B01A7CF80917101909172018C
:100A7000019711F461E001C060E080912B019BCFF0
:100A800061E080912F010E94910884E090E00E9433
:100A90005F0A0E94E7020E949B079B01AC016093E2
:100AA0006301709364018093650190936601809166
:100AB0006D0190916E01019709F053C0809167011B
:100AC00090916801A0916901B0916A01281B390BCE
:100AD0004A0B5B0B80916B0190916C01AA2797FDEB
:100AE000A095BA2F281739074A075B07A0F16FEFC7
:100AF00070E080911D010E941B08E0906301F0905E
:100B000064010091650110916601809167019091E7
:100B10006801A0916901B0916A01A8019701281BA1
:100B2000390B4A0B5B0B80916B0190916C01880F24
:100B3000991FAA2797FDA095BA2F281739074A07AA
:100B40005B0778F0E0926701F09268010093690119
:100B500010936A0106C060E070E080911D010E9460
:100B60001B081F910F91FF90EF9008950E94E107DD
:100B70000E9401020E942A03FDCF87E391E0909337
:100B80007C0180937B010895862F0E94610908955E
:100B90000E947A0908950E9469090895CB01BA015B
:100BA0000E94280908950F931F93CF93DF938C0120
:100BB000EB0109C02196D801ED91FC910190F081E3
:100BC000E02DC801099568816623A1F7DF91CF91D7
:100BD0001F910F9108950F931F938C01DC01ED91EC
:100BE000FC910190F081E02D6DE00995D801ED9127
:100BF000FC910190F081E02D6AE0C80109951F91F8
:100C00000F9108952F923F924F925F926F927F9231
:100C10008F929F92AF92BF92CF92DF92EF92FF920C
:100C20000F931F93DF93CF93CDB7DEB7A0970FB687
:100C3000F894DEBF0FBECDBF1C016A017B014115D8
:100C400051056105710549F4DC01ED91FC910190BC
:100C5000F081E02D60E3099554C088249924540163
:100C6000422E55246624772401E010E00C0F1D1F4E
:100C7000080D191DC701B601A30192010E94080ABF
:100C8000F80160830894811C911CA11CB11CC70150
:100C9000B601A30192010E94080AC901DA016C01A0
:100CA0007D01C114D104E104F104F1F681E0E82EE4
:100CB000F12CEC0EFD1EE80CF91C3E010894611CA1
:100CC000711CD501C4010197A109B1096C01C818B3
:100CD000D90814C0F601EE0DFF1D60816A3010F4D2
:100CE000605D01C0695CD101ED91FC910190F081E2
:100CF000E02DC10109950894E108F1086E147F0404
:100D000049F7A0960FB6F894DEBF0FBECDBFCF91C6
:100D1000DF911F910F91FF90EF90DF90CF90BF90E8
:100D2000AF909F908F907F906F905F904F903F908B
:100D30002F900895EF92FF920F931F93CF93DF931D
:100D4000EC017A018B0177FF0FC0E881F9810190F6
:100D5000F081E02D6DE2099510950095F094E094F6
:100D6000E11CF11C011D111D2AE0B801A701CE01F3
:100D70000E940206DF91CF911F910F91FF90EF909B
:100D800008950F931F938C01AB01662757FD609563
:100D9000762F0E949A06C8010E94EB051F910F91C1
:100DA00008951F920F920FB60F9211242F933F9325
:100DB0004F935F936F937F938F939F93AF93BF9363
:100DC000EF93FF9380917D0190917E01892B29F013
:100DD000E0917D01F0917E010995FF91EF91BF9126
:100DE000AF919F918F917F916F915F914F913F91C3
:100DF0002F910F900FBE0F901F9018951F920F927A
:100E00000FB60F9211242F933F934F935F936F93DD
:100E10007F938F939F93AF93BF93EF93FF938091B3
:100E20007F0190918001892B29F0E0917F01F09161
:100E300080010995FF91EF91BF91AF919F918F91A3
:100E40007F916F915F914F913F912F910F900FBEC6
:100E50000F901F9018951F920F920FB60F921124AA
:100E60002F938F939F93AF93BF9380918101909124
:100E70008201A0918301B09184010196A11DB11D51
:100E80008093810190938201A0938301B0938401A8
:100E90008091850190918601A0918701B091880190
:100EA0008050904CAF4FBF4F809385019093860147
:100EB000A0938701B093880127C08091850190910C
:100EC0008601A0918701B091880180589E43A0407F
:100ED000B0408093850190938601A0938701B093E1
:100EE00088018091890190918A01A0918B01B09134
:100EF0008C010196A11DB11D8093890190938A01F7
:100F0000A0938B01B0938C01809185019091860113
:100F1000A0918701B091880181589E43A040B040C4
:100F200060F6BF91AF919F918F912F910F900FBE5F
:100F30000F901F9018958FB7F894209189013091E8
:100F40008A0140918B0150918C018FBFB901CA0178
:100F50000895EF92FF920F931F937B018C018FB73F
:100F6000F8944091890150918A0160918B017091B0
:100F70008C018FBF2FB7F8948091890190918A01DD
:100F8000A0918B01B0918C012FBF841B950BA60BF8
:100F9000B70BE816F9060A071B0760F71F910F91B8
:100FA000FF90EF900895019759F0FC01EE0FFF1F9D
:100FB000EE0FFF1F32978FB7F8943197F1F78FBF7D
:100FC0000895789484B5826084BD84B5816084BDC1
:100FD00085B5826085BD85B5816085BDEEE6F0E0B2
:100FE000808181608083E1E8F0E08081826080839D
:100FF000808181608083E0E8F0E08081816080838F
:10100000E1EBF0E0808184608083E0EBF0E08081C0
:1010100081608083EAE7F0E0808184608083808162
:10102000826080838081816080838081806880830A
:101030001092C10008951F93CF93DF93182FEB01F7
:1010400061E00E947308E12FF0E0E156FF4F8491C8
:10105000833051F480918000806880938000D09329
:101060008900C09388003BC0843051F48091800097
:10107000806280938000D0938B00C0938A002FC041
:10108000813039F4209729F184B5806884BDC7BDCB
:1010900026C0823039F42097E1F084B5806284BDA7
:1010A000C8BD1DC0863041F48091B0008068809337
:1010B000B000C093B30013C0873041F48091B000FA
:1010C00080628093B000C093B40009C0C038D105DD
:1010D00014F460E001C061E0812F0E949108DF916B
:1010E000CF911F910895282F30E0C90185579F4F58
:1010F000FC01949129583F4FF9018491882381F094
:10110000E82FF0E0E859FF4FE491F0E0662329F47E
:10111000808190958923808308958081892B8083A5
:101120000895482F50E0CA0181569F4FFC01249139
:10113000CA0185579F4FFC01949149585F4FFA01AE
:1011400034913323C1F1222331F1233021F48091F2
:1011500080008F7705C0243031F4809180008F7D2E
:101160008093800018C0213019F484B58F7704C0B3
:10117000223021F484B58F7D84BD0DC0263021F44A
:101180008091B0008F7705C0273029F48091B0009E
:101190008F7D8093B000E32FF0E0E359FF4FE4919F
:1011A000F0E0662329F48081909589238083089557
:1011B0008081892B80830895482F50E0CA01815691
:1011C0009F4FFC012491CA0185579F4FFC019491C8
:1011D00049585F4FFA013491332319F420E030E08D
:1011E00035C0222331F1233021F4809180008F77A4
:1011F00005C0243031F4809180008F7D8093800081
:1012000018C0213019F484B58F7704C0223021F43E
:1012100084B58F7D84BD0DC0263021F48091B0004F
:101220008F7705C0273029F48091B0008F7D80939F
:10123000B000E32FF0E0EE58FF4FE491F0E0808142
:1012400020E030E0892311F021E030E0C901089569
:10125000EF92FF920F931F937B018C0122E030E00D
:1012600040E050E00E942A0A205C3D4B404F5F4F17
:10127000CA01B901A80197010E942A0AC901DA012D
:101280000197A109B109292F3A2F4B2F552747FD67
:101290005A950196A11DB11D2093C50081508093E0
:1012A000C400E1ECF0E0808180618083808188600F
:1012B00080838081806880831F910F91FF90EF90E1
:1012C0000895982F8091C00085FFFCCF9093C600B1
:1012D000089580918D0190918E0180589F4F2091AB
:1012E0008F0130919001821B930B60E870E00E94A7
:1012F000F509089540918F015091900180918D01E1
:1013000090918E018417950719F42FEF3FEF0FC0CE
:10131000FA01EF56FE4F2081CA01019660E870E0A5
:101320000E94F5099093900180938F0130E0C901EC
:1013300008951F920F920FB60F9211242F933F938F
:101340004F935F936F937F938F939F93AF93BF93CD
:10135000EF93FF934091C600E0918D01F0918E01D3
:10136000CF01019660E870E00E94F5099C01809130
:101370008F01909190012817390739F0EF56FE4FF1
:10138000408330938E0120938D01FF91EF91BF91A7
:10139000AF919F918F917F916F915F914F913F910D
:1013A0002F910F900FBE0F901F901895629FD00144
:1013B000739FF001829FE00DF11D649FE00DF11D10
:1013C000929FF00D839FF00D749FF00D659FF00DBF
:1013D0009927729FB00DE11DF91F639FB00DE11DAC
:1013E000F91FBD01CF011124089597FB092E07268F
:1013F0000AD077FD04D049D006D000201AF47095A9
:1014000061957F4F0895F6F7909581959F4F0895C8
:10141000A1E21A2EAA1BBB1BFD010DC0AA1FBB1FF8
:10142000EE1FFF1FA217B307E407F50720F0A21B6A
:10143000B30BE40BF50B661F771F881F991F1A94D7
:1014400069F760957095809590959B01AC01BD0101
:10145000CF01089597FB092E05260ED057FD04D025
:10146000D7DF0AD0001C38F450954095309521956F
:101470003F4F4F4F5F4F0895F6F7909580957095C9
:1014800061957F4F8F4F9F4F0895AA1BBB1B51E162
:1014900007C0AA1FBB1FA617B70710F0A61BB70BE4
:1014A000881F991F5A95A9F780959095BC01CD0189
:1014B0000895EE0FFF1F0590F491E02D099491110E
:1014C000089581568A5108F4805285580895F894F9
:0214D000FFCF4C
:1014D200486F6C612C20736F7920656C20726F628B
:1014E2006F74206E756D65726F200008000B00042A
:1014F2000002000E000F001000110003000500079B
:0A15020000090A00000000C4050003
:00000001FF
